:1000000012C02CC02BC02AC029C028C027C026C0BF
:1000100025C024C023C022C021C020C01FC01EC0D4
:100020001DC01CC01BC011241FBECFE5D4E0DEBF25
:10003000CDBF10E0A0E6B0E0E8EFFAE002C0059026
:100040000D92A43DB107D9F710E0A4EDB0E001C0D6
:100050001D92AC3DB107E1F7D9D24CC5D1CF14BA4E
:1000600017BA11BA80EF81BB87B3836087BBBA9A96
:10007000089586B1876886B9089567E070E0ACD4CA
:1000800087B9369A3699FECF24B135B1C9010895A2
:10009000C09A83E08A95F1F70000C09880E18A95C4
:1000A000F1F700C00895982F991F9927991F9295ED
:1000B000907F86FD906285FD906484FD906883FD4D
:1000C000916082FD926081FD946080FD986082B3B2
:1000D0008F7082BB903118F482B3929501C082B3C5
:1000E000907F982B92BB662311F0C19A01C0C198F2
:1000F000CFDF08951F93182F807F60E0D4DF812F1A
:100100008F7060E0D0DF1F910895982F862F933075
:1001100031F0943031F0923031F4815405C0815780
:1001200003C0815301C08158E5DF8DEE92E0019755
:10013000F1F700C00000089581E0DCDF8DEE92E071
:100140000197F1F700C00000089583ED90E3019757
:10015000F1F700C0000080E360E0A5DF87E893E1ED
:100160000197F1F700C0000080E360E09CDF92E4BB
:100170009A95F1F700C080E360E095DF87EA91E6A9
:100180000197F1F700C0000080E260E08CDF89E6B3
:1001900098E10197F1F700C000008CE2ABDF89E63F
:1001A00098E10197F1F700C000008CE0A3DF89E639
:1001B00098E10197F1F700C0000086E09BDF83E241
:1001C00094EF0197F1F700C0000008951F93182FD6
:1001D000807F61E068DF812F8F7061E064DF1F91B5
:1001E0000895EF92FF92CF93DF93E82EE7017E010F
:1001F000F92EE70105C0EADF96E09A95F1F700C015
:1002000089918823C1F7DF91CF91FF90EF900895F6
:100210009C01FB0197FF05C0309521953F4F8DE272
:1002200009C0009731F480E28093D40020E030E0F0
:100230000EC08BE28093D40083E0293E38073CF067
:10024000C90168EE73E0C8D3805D8093D400C90112
:1002500068EE73E0C1D364E670E0BED3262F205D64
:100260002093D5006AE070E0B7D3605D6093D6005C
:10027000805DE130F10531F49EE29093D7008093E8
:10028000D80004C08093D7001092D8001092D900F3
:10029000203319F480E28093D50084ED90E0089536
:1002A00097FF05C0909581959F4F2DE209C000975B
:1002B00031F480E28093D40080E090E003C02BE230
:1002C0002093D40060E177E287D3605D6093D5002E
:1002D00068EE73E081D3605D6093D60064E670E001
:1002E0007BD3605D6093D7006AE070E075D3605D9A
:1002F0006093D800805D8093D9001092DA0084ED7D
:1003000090E008958AE090E0CBD3AA2797FDA095CE
:10031000BA2F8093CF009093D000A093D100B093D8
:10032000D2008F3F2FEF92072FEFA2072FEFB207D8
:1003300029F484ED9EEFAFEFBFEF19C08C302EEFA4
:1003400092072FEFA2072FEFB2072CF48CE09EEF5D
:10035000AFEFBFEF0CC08D392FEF92072FEFA20741
:100360002FEFB20764F08CE99FEFAFEFBFEF809300
:10037000CF009093D000A093D100B093D20084E13D
:1003800090E08ED3AA2797FDA095BA2F8093CB003B
:100390009093CC00A093CD00B093CE008F3F2FEF71
:1003A00092072FEFA2072FEFB20729F48CE291E01A
:1003B000A0E0B0E00CC0853F21E0920720E0A2075A
:1003C00020E0B2076CF084EF91E0A0E0B0E0809311
:1003D000CB009093CC00A093CD00B093CE000895B5
:1003E00084369105A105B10564F484E690E0A0E0AF
:1003F000B0E08093CB009093CC00A093CD00B0935D
:10040000CE000895CF93DF9397DE81E061E07DDE3B
:1004100080E690E0E6DE8FE996E8A1E0815090402A
:10042000A040E1F700C00000C0E0D0E081E06CE057
:100430006CDE8091CF009091D00060E070E0E8DE4B
:10044000D0DEAFE4B3EC1197F1F700C00000829B5F
:1004500002C021961DC08091CF009091D000A09144
:10046000D100B091D2008D302EEF92072FEFA2076E
:100470002FEFB2075CF00196A11DB11D8093CF0054
:100480009093D000A093D100B093D200C0E0D0E010
:1004900083991DC08091CF009091D000A091D10090
:1004A000B091D2008C392FEF92072FEFA2072FEFD8
:1004B000B2070CF0B9CF0197A109B1098093CF0021
:1004C0009093D000A093D100B093D200ADCFC431AF
:1004D000D1050CF4ABCF82E061E017DE8DE690E051
:1004E00080DE8FE996E8A1E081509040A040E1F7DE
:1004F00000C00000C0E0D0E082E06CE006DE809149
:10050000CB009091CC0060E070E082DE6ADEAFE468
:10051000B3EC1197F1F700C00000839B02C0219655
:100520001DC08091CB009091CC00A091CD00B091E6
:10053000CE00843F21E0920720E0A20720E0B2072E
:100540005CF40196A11DB11D8093CB009093CC006B
:10055000A093CD00B093CE00C0E0D0E082991AC045
:100560008091CB009091CC00A091CD00B091CE00B5
:1005700085369105A105B1050CF4BCCF0197A10901
:10058000B1098093CB009093CC00A093CD00B093A1
:10059000CE00B0CFC431D1050CF4AECF6091CF0006
:1005A0007091D0008AE090E080D26091CB00709191
:1005B000CC0084E190E079D2A5DEBEDD81E062E08E
:1005C000A4DD8AE790E00DDE82E061E09EDD8091AF
:1005D000CF009091D00060E070E01ADE02DE82E091
:1005E0006AE093DD8091CB009091CC0060E070E0F8
:1005F0000FDEF7DD8FE79AE1A6E081509040A04042
:10060000E1F700C00000DF91CF9108952F923F9253
:100610004F925F926F927F928F929F92AF92BF9212
:10062000CF92DF92EF92FF920F931F93DF93CF93BE
:1006300000D00F92CDB7DEB787EA91E60197F1F7C8
:1006400000C000000CDDC29A8FE996E8A1E081505D
:100650009040A040E1F700C0000077DD53DEA3ED3D
:10066000B0E31197F1F700C0000066DD86E890E086
:10067000B8DD82E063E049DD87E990E0B2DD83E048
:1006800063E043DD84EA90E0ACDD84E063E03DDDDF
:100690008FEA90E0A6DD80E090E020B32C702C3053
:1006A00019F0B0DE8EE190E0E7EAF1E63197F1F77C
:1006B00000C0000001968E3191057CF3DADC3CDD50
:1006C00088B3F4E08F2788BB83EC99E00197F1F7BA
:1006D00000C0000081E061E018DD8AE090E0EE24D7
:1006E000FF2487016C0180E090E0C7DCAA2797FD1A
:1006F000A095BA2FE80EF91E0A1F1B1FA3ECB9E044
:100700001197F1F700C000000894C108D108C11486
:10071000D10449F7C801B7012CEE3FEF4FEF5FEF6F
:100720006ED1D22EC32EB42E552EC90161E070E0D9
:100730006FDD57DD8CEB90E054DDE3ECF9E03197B1
:10074000F1F700C0000081E06AE0DFDC8AE090E0C1
:10075000EE24FF2487013C0181E090E08EDCAA2793
:1007600097FDA095BA2FE80EF91E0A1F1B1F83ECF8
:1007700099E00197F1F700C0000008946108710842
:100780006114710449F7C801B70124E130E040E089
:1007900050E035D1A22E39834A835B83C90161E0E1
:1007A00070E036DD1EDD8CEB90E01BDDA3ECB9E0E4
:1007B0001197F1F700C0000082E061E0A6DC8AE05A
:1007C00090E0EE24FF2487013C0182E090E055DCBC
:1007D000AA2797FDA095BA2FE80EF91E0A1F1B1F26
:1007E000E3ECF9E03197F1F700C0000008946108EC
:1007F00071086114710449F7C801B7016B5F734157
:100800008040904097FF03C060E070E0CB012091F2
:10081000CF003091D0004091D1005091D200BDD096
:1008200020E137E240E050E0EAD039014A01C90155
:1008300061E070E0EDDCD5DC8EEB90E0D2DC83ECA7
:1008400099E00197F1F700C0000082E06AE05DDC0A
:100850008AE090E0EE24FF2487011C0183E090E011
:100860000CDCAA2797FDA095BA2FE80EF91E0A1FE7
:100870001B1FA3ECB9E01197F1F700C0000008942A
:10088000210831082114310449F7C801B7016B5F11
:1008900073418040904097FF03C060E070E0CB015F
:1008A0002091CB003091CC004091CD005091CE00F2
:1008B00074D020E137E240E050E0A1D079018A0114
:1008C000C90161E070E0A4DC8CDC8EEB90E089DC97
:1008D000E3ECF9E03197F1F700C0000083E061E05C
:1008E00014DCC401B3012D2D3C2D4B2D552D55D0BD
:1008F00026EF3FEF4FEF5FEF82D019012A01C901C8
:1009000061E070E085DC6DDC80EC90E06ADC83E027
:100910006AE0FBDBC801B7012A2D39814A815B817E
:100920003CD02AE030E040E050E069D059016A0153
:10093000C90161E070E06CDC54DC80EC90E051DCDB
:1009400084E063E0E2DBD801C70186199709A809B2
:10095000B90961E070E05CDC44DC82EC90E041DCF1
:1009600084E061E0D2DB85EC90E03BDC84E06BE08E
:10097000CCDBD601C50182199309A409B50961E050
:1009800070E046DC2EDC80EC90E02BDC84E06BE059
:10099000BCDB89EC90E025DC93CE629FD001739F95
:1009A000F001829FE00DF11D649FE00DF11D929F0B
:1009B000F00D839FF00D749FF00D659FF00D99274A
:1009C000729FB00DE11DF91F639FB00DE11DF91F6E
:1009D000BD01CF011124089597FB092E07260AD0E7
:1009E00077FD04D027D006D000201AF470956195C9
:1009F0007F4F0895F6F7909581959F4F089597FB47
:100A0000092E05260ED057FD04D028D00AD0001C90
:100A100038F450954095309521953F4F4F4F5F4F9B
:100A20000895F6F790958095709561957F4F8F4F5B
:100A30009F4F0895AA1BBB1B51E107C0AA1FBB1FF4
:100A4000A617B70710F0A61BB70B881F991F5A955A
:100A5000A9F780959095BC01CD010895A1E21A2EC9
:100A6000AA1BBB1BFD010DC0AA1FBB1FEE1FFF1F52
:100A7000A217B307E407F50720F0A21BB30BE40BA2
:100A8000F50B661F771F881F991F1A9469F76095E9
:100A90007095809590959B01AC01BD01CF010895A3
:100AA000A8E1B0E042E050E006C00196272F12D046
:100AB00010C0DC01CB01FC01E199FECF06C0FFBBF9
:100AC000EEBBE09A31960DB20D9241505040B8F70E
:100AD0000895262FE199FECF9FBB8EBBE09A019728
:100AE0000DB2021631F02DBB0FB6F894E29AE19ADE
:080AF0000FBE0895F894FFCF3A
:100AF8004E656761746976654D463A2000506F739C
:100B080069746976654D463A20005341564544203C
:100B180041532E2E2E0053696D706C666420424935
:100B28002D504F4C41520020564F4C542D4D45549A
:100B3800455220002020414D4D455445522000206B
:100B4800574154542D4D45544552200056004100FC
:100B5800570041200053554D00200036010000CABF
:040B6800FEFFFF008D
:00000001FF
